:100000000C943400189500000C94D8091895000041
:10001000189500001895000018950000189500002C
:10002000189500000C94570A1895000018950000C8
:10003000189500000C94C30818950000189500004E
:1000400018950000189500001895000018950000FC
:1000500018950000189500001895000018950000EC
:1000600018950000189500008FEF8DBFC0EEE0EBF3
:100070004E2E84E08EBFD4E0F4E05F2EA89584B7C6
:10008000082E877F84BF88E1992780936000909332
:100090006000EEEFF3E0A0E0B1E088278D933197A8
:1000A000E9F781E08093C40080E08093C50088E197
:1000B0008093C1000E94210B662487E08093B100E9
:1000C00080E08093B0007091700071607093700058
:1000D00080916900837F84608093690080E08093D1
:1000E000800081E0809381005298539854985A9AE6
:1000F0005B9A5C9A249A3C9A3D9A449A459A7894E1
:1001000084E690E00E94F30B80E08093120181E08E
:10011000809313012C9A0E94D10CE0E0F0E0ADE056
:10012000B1E092E00E94BA0C0E940608E2E0F0E022
:10013000A5E2B1E091E00E94BA0CE3E0F0E0A0E1BA
:10014000B1E091E00E94BA0CE4E0F0E0A1E1B1E09E
:1001500091E00E94BA0CE5E0F0E0A7E2B1E091E0A6
:100160000E94BA0CE6E0F0E0A8E2B1E091E00E9463
:10017000BA0CE7E0F0E0A9E2B1E091E00E94BA0C2D
:10018000E8E0F0E0ABE0B1E092E00E94BA0C0E943F
:1001900097080E94AA080E9458088CE00E946F0BE2
:1001A0000E94060BE0E5FAE10E94FD0AE8E5FAE1AB
:1001B0000E94FD0A00912801033011F00C94E60022
:1001C0000E94040BEEE5FAE10E94FD0A4C990C94A2
:1001D000F4000E94060BEEE6FAE10E94FD0A4C9B39
:1001E0000C94EF000E947F05E1E0F0E00E94180B04
:1001F0000E940608E0E0F0E0ADE0B1E092E07BE7CD
:100200000E94A90C0E941807A5E2B1E00C9100FB26
:1002100016F00C943D010E9445088FE710E10E9402
:10022000150B00912801023011F00C941B018FEB8B
:1002300018E00E94150B00912A01013011F00C9476
:100240002701E6E7FAE10E94FD0A0C943D01AFE0C8
:10025000B1E00C9106FB16F00C943201E8E7FAE1EC
:100260000E94FD0AAFE0B1E00C9106FB16F40C947D
:100270003D01EAE7FAE10E94FD0AA0E0B1E08C91BD
:1002800087FB16F00C9446010C947101A0E0B1E0DC
:100290008C9186FB16F00C944F010C9499014C99AB
:1002A0000C94580188EC90E00E94F30B0C94C2016E
:1002B0000E94E80A082F0B3781E009F080E08F9355
:1002C0000E94E80A082F0C3781E009F080E09F9136
:1002D000892B882311F40C946F010C94001C0C944E
:1002E0000401709100017F7770930001ADE0B1E0EF
:1002F0000D911C91A0E1B1E04D915527040F151F00
:10030000ADE0B1E00D931C93ADE0B1E00D911C9117
:1003100000365DE6150718F011F00C9491010C946D
:10032000970180E89CE0ADE0B1E08D939C930C9444
:10033000F800709100017F7B70930001ADE0B1E0A7
:100340000D911C91A0E1B1E04D915527041B150BB7
:10035000ADE0B1E00D931C93ADE0B1E04D915C9147
:1003600000E81CE00417150718F011F00C94BA010E
:100370000C94C00180E69DE6ADE0B1E08D939C93C6
:100380000C94F8000E94060B00911201013011F04C
:100390000C94DC01ECE7FAE10E94FD0A00912801CF
:1003A000033011F00C94DA010E94040BEAE8FAE140
:1003B0000E94FD0A0C944402023011F00C94F201E8
:1003C000EAE8FAE10E94FD0A00912801033011F0E9
:1003D0000C94F0010E94040BEAE9FAE10E94FD0A84
:1003E0000C944402033011F00C940802EAE9FAE19B
:1003F0000E94FD0A00912801033011F00C940602BE
:100400000E94040BE2EAFAE10E94FD0A0C94440205
:10041000043011F00C941E02E2EAFAE10E94FD0A97
:1004200000912801033011F00C941C020E94040B6F
:10043000E2EBFAE10E94FD0A0C944402053011F04F
:100440000C943402E2EBFAE10E94FD0A00912801CB
:10045000033011F00C9432020E94040BECEBFAE131
:100460000E94FD0A0C944402ECEBFAE10E94FD0AA2
:1004700000912801033011F00C9444020E94040BF7
:10048000ECE7FAE10E94FD0AA0E0B1E08C9187FB65
:1004900016F00C946302A2E1B1E08C918F5F8C9313
:1004A00000911201053018F011F00C9459020C94CF
:1004B0005C0280E080931201709100017F7770935D
:1004C00000010C94C201A0E0B1E08C9186FB16F013
:1004D0000C9482028091120181508093120100914C
:1004E0001201053018F011F00C9478020C947B0284
:1004F00085E080931201709100017F7B7093000171
:100500000C94C2014C990C94B50288EC90E00E94C6
:10051000F30B00911201013011F00C9493020C9432
:10052000B7020C94B502023011F00C949B020C94AB
:1005300040030C94B502033011F00C94A3020C9408
:10054000B6030C94B502043011F00C94AB020C9479
:1005500014040C94B502053011F00C94B3020C9401
:10056000D5040C94B5020C94F8000C9444020E943B
:10057000060B00912801033011F00C94C502ECE742
:10058000FAE10E94FD0A0E94040B0DE710E0A0E1D1
:10059000B1E04D9155270E94020CA9E0B1E00D9306
:1005A0001C93A9E0B1E00D911C91A1E1B1E04D9146
:1005B00055270E94020CA9E0B1E00D931C93A8E915
:1005C000B4E0E9E0F1E00E94470C0E94F50AECEC8F
:1005D000FAE10E94FD0AA0E0B1E08C9187FB16F0E1
:1005E0000C94F4020C941003A0E0B1E08C9186FB13
:1005F00016F00C94FD020C9429034C990C940E03F4
:10060000E3E0F0E0A0E1B1E091E07BE70E94A90C1B
:1006100088EC90E00E94F30B0C94C2010C94EB0266
:10062000709100017F7770930001A0E1B1E00C911F
:1006300042E0049F0C9200911001003418F011F078
:100640000C9424030C94270381E0809310010C94F4
:10065000B702709100017F7B70930001009110013F
:10066000013011F00C94370380E880931001A0E171
:10067000B1E00C9142E00E94C10C0C930C94B702C3
:100680000E94060B00912801033011F00C944E03D8
:10069000EAE8FAE10E94FD0A0E94040B00911101B0
:1006A0000A3010F00C945803E0EDFAE10E94FD0AC4
:1006B000A8E9B4E0E1E1F1E00E94560C0E94F50ADD
:1006C000E2EDFAE10E94FD0AA0E0B1E08C9187FB27
:1006D00016F00C946D030C948903A0E0B1E08C91AA
:1006E00086FB16F00C9476030C94A1034C990C94A1
:1006F0008703E4E0F0E0A1E1B1E091E07BE70E9454
:10070000A90C88EC90E00E94F30B0C94C2010C94AD
:100710006403709100017F7770930001A1E1B1E063
:100720008C918F5F8C93009111010A3018F011F0B9
:100730000C949C030C949F0381E0809311010C9412
:100740004003709100017F7B70930001A1E1B1E053
:100750008C9181508C9300911101013010F00C9418
:10076000B4038AE0809311010C94400382E390E08B
:100770000E94F30B0E94060B00912801033011F038
:100780000C94C803EAE9FAE10E94FD0A0E94040BF6
:10079000A5E2B1E00C9100FB16F40C94D503E8ED52
:1007A000FAE10E94FD0A0C94D903ECEDFAE10E94F3
:1007B000FD0AA0E0B1E08C9187FB16F00C94ED03EC
:1007C000A5E2B1E08C9191E089278C9370910001B2
:1007D0007F77709300010C94B603A0E0B1E08C9198
:1007E00086FB16F00C940104A5E2B1E08C9191E037
:1007F00089278C93709100017F7B709300010C948A
:10080000B6034C990C941204E2E0F0E0A5E2B1E0EA
:1008100091E07BE70E94A90C88EC90E00E94F30B2A
:100820000C94C2010C94D90382E390E00E94F30B74
:100830000E94060B00912801033011F00C9426044D
:10084000E2EAFAE10E94FD0A0E94040B00912701EE
:10085000013011F00C943304E8EDFAE10E94FD0A36
:100860002C980C944704023011F00C943E04ECEDEB
:10087000FAE10E94FD0A2C9A0C944704033011F00F
:100880000C944704E0EEFAE10E94FD0A2C9AA0E0E5
:10089000B1E08C9187FB16F00C946604A7E2B1E0FE
:1008A0008C918F5F8C9300912701033018F011F029
:1008B0000C945C040C945F0481E080932701709198
:1008C00000017F77709300010C949D04A0E0B1E0DB
:1008D0008C9186FB16F00C94820480912701815044
:1008E0008093270100912701013010F00C947B04C4
:1008F00083E080932701709100017F7B709300015A
:100900000C949D044C990C949B04E2E0F0E0A5E269
:10091000B1E091E07BE70E94A90CE5E0F0E0A7E2FE
:10092000B1E091E07BE70E94A90C88EC90E00E9486
:10093000F30B0C94C2010C94470400912701013081
:1009400011F00C94B104E894A5E2B1E08C9182F925
:100950008C93E894A5E2B1E08C9181F98C930C948E
:10096000D304023011F00C94C304E894A5E2B1E082
:100970008C9182F98C936894A5E2B1E08C9181F915
:100980008C930C94D304033011F00C94D30468942A
:10099000A5E2B1E08C9182F98C936894A5E2B1E074
:1009A0008C9181F98C930C9414040E9458080E9435
:1009B000060B00912801033011F00C94E504ECE7DC
:1009C000FAE10E94FD0A0E94040B0AE010E0ABE08D
:1009D000B1E04D915C910E94020CA9E0B1E00D9351
:1009E0001C93A8E9B4E0E9E0F1E00E94470C0E9402
:1009F000F50AECECFAE10E94FD0A8FE718E00E948C
:100A0000150B00912A01013011F00C940D05E6E759
:100A1000FAE10E94FD0A0C941105E0EDFAE10E9452
:100A2000FD0AA0E0B1E08C9187FB16F00C941A054A
:100A30000C943605A0E0B1E08C9186FB16F00C9486
:100A400023050C945C054C990C943405E8E0F0E027
:100A5000ABE0B1E092E07BE70E94A90C88EC90E06B
:100A60000E94F30B0C94C2010C94110570910001CB
:100A70007F7770930001ABE0B1E00D911C9141E0F4
:100A800050E0040F151FABE0B1E00D931C93ABE0F9
:100A9000B1E00D911C91083E53E0150718F011F0DC
:100AA0000C9454050C945A0584EF91E0ABE0B1E04E
:100AB0008D939C930C94D504709100017F7B70936F
:100AC0000001ABE0B1E00D911C9141E050E0041B4E
:100AD000150BABE0B1E00D931C93ABE0B1E00D91D1
:100AE0001C91043F51E0150710F00C947D0588EE31
:100AF00093E0ABE0B1E08D939C930C94D5040E94FD
:100B0000060B00911301013011F00C949905EEE6EB
:100B1000FAE10E94FD0A00912801033011F00C94C3
:100B200097050E94040BE6EEFAE10E94FD0A0C9480
:100B3000BF05023011F00C94AF05E6EEFAE10E9419
:100B4000FD0A00912801033011F00C94AD050E94BC
:100B5000040BE4EFFAE10E94FD0A0C94BF05E4EFF8
:100B6000FAE10E94FD0A00912801033011F00C9473
:100B7000BF050E94040BEEE6FAE10E94FD0AA0E028
:100B8000B1E08C9187FB16F00C94DE05A3E1B1E097
:100B90008C918F5F8C9300911301023018F011F04B
:100BA0000C94D4050C94D70580E0809313017091C8
:100BB00000017F77709300010C947F05A0E0B1E005
:100BC0008C9186FB16F00C94FD05809113018150E9
:100BD0008093130100911301023018F011F00C946E
:100BE000F3050C94F60582E08093130170910001E7
:100BF0007F7B709300010C947F054C990C94180630
:100C000088EC90E00E94F30B00911301013011F089
:100C10000C940E060C941A060C941806023011F06F
:100C20000C9416060C949C060C9418060C94F80070
:100C30000C94BF0582E390E00E94F30B0E94060B28
:100C400000912801033011F00C942C06EEE6FAE135
:100C50000E94FD0A0E94040B00912801013011F04E
:100C60000C943806EEEFFAE10E94FD0A0C944A0655
:100C7000023011F00C944206E6E0FBE10E94FD0A0E
:100C80000C944A06033011F00C944A06EEE0FBE1A6
:100C90000E94FD0AA0E0B1E08C9187FB16F00C9455
:100CA0006906A8E2B1E08C918F5F8C9300912801D6
:100CB000033018F011F00C945F060C94620681E08A
:100CC00080932801709100017F77709300010C944C
:100CD0009806A0E0B1E08C9186FB16F00C94850696
:100CE00080912801815080932801009128010130D2
:100CF00010F00C947E0683E080932801709100012F
:100D00007F7B709300010C9498064C990C94960686
:100D1000E6E0F0E0A8E2B1E091E07BE70E94A90CF8
:100D200088EC90E00E94F30B0C947F050C944A062B
:100D30000E9497080C941A0682E390E00E94F30B3D
:100D40000E94060B00912801033011F00C94AE06AE
:100D5000E6EEFAE10E94FD0A0E94040BE6E1FBE1E7
:100D60000E94FD0A00912901013011F00C94BE0689
:100D7000ECE1FBE10E94FD0A0C94C606023011F082
:100D80000C94C606E4E2FBE10E94FD0AA0E0B1E09B
:100D90008C9187FB16F00C94E506A9E2B1E08C91EA
:100DA0008F5F8C9300912901023018F011F00C94A0
:100DB000DB060C94DE0681E080932901709100012E
:100DC0007F77709300010C941407A0E0B1E08C9140
:100DD00086FB16F00C9401078091290181508093C5
:100DE000290100912901013010F00C94FA0682E0EB
:100DF00080932901709100017F7B709300010C9416
:100E000014074C990C941207E7E0F0E0A9E2B1E076
:100E100091E07BE70E94A90C88EC90E00E94F30B24
:100E20000C947F050C94C6060E94AA080C949C069C
:100E3000ADE0B1E00D911C9122273327A1E1B1E093
:100E40004C915527662777270E940C0CA1E0B1E052
:100E50000D931D932D933D93A1E0B1E00D911C9155
:100E600048E050E00E94C70AA7E0B1E00D931C9350
:100E7000A7E0B1E00D911C914DE750E00E94020CFB
:100E8000A7E0B1E00D931C93A1E0B1E00D911D919D
:100E90002D913C9148E050E060E070E00E94930B9F
:100EA000A1E0B1E04D935D936D937D93A1E0B1E03E
:100EB0008D919C91A5E0B1E08D939C930E94060BCF
:100EC000A4E1B1E088278C93A5E0B1E00D911C91DD
:100ED000083E53E0150710F00C949807A4E1B1E028
:100EE000E0EDFAE10E942F0CA5E0B1E00D911C911C
:100EF000043650E0150710F00C949807A4E1B1E017
:100F00000E94E10AE0EDFAE10E942F0CA5E0B1E0B9
:100F10000D911C910A3050E0150710F00C949807C1
:100F2000A4E1B1E00E94E10AE0EDFAE10E942F0C99
:100F3000A4E1B1E00E94E10AE5E0F1E00E94470C83
:100F4000A4E1B1E00E94E10AEEE2FBE10E942F0C75
:100F5000A7E0B1E00D911C91043650E0150710F0A8
:100F60000C94CC07A4E1B1E00E94E10AE0E3FBE1CC
:100F70000E942F0CA7E0B1E00D911C910A3050E0C7
:100F8000150710F00C94CC07A4E1B1E00E94E10A2F
:100F9000E0E3FBE10E942F0CA4E1B1E00E94E10A32
:100FA000E7E0F1E00E94470CA4E1B1E00E94E10A11
:100FB000E2E3FBE10E942F0CA4E1B1E00E94F70AFA
:100FC00000912801033011F40C94E70708950E9462
:100FD000040BE6E3FBE10E94FD0A0DE710E0A0E14F
:100FE000B1E04D9155270E94020CA9E0B1E00D93AC
:100FF0001C93A8E9B4E0E9E0F1E00E94470C0E94EC
:10100000F50AECECFAE10E94FD0A08950E94D60C64
:1010100012EC0E94EE0CADE0B1E011968C91A9E0CB
:10102000B1E08D9388278C93A9E0B1E01C910E94D8
:10103000EE0CADE0B1E08C91A9E0B1E08D93882792
:101040008C93A9E0B1E01C910E94EE0C8EEC90E034
:10105000A9E0B1E08D939C93A9E0B1E01C910E94BE
:10106000EE0C80E090E0A9E0B1E08D939C93A9E0C4
:10107000B1E01C910E94EE0C0E94E50C62FAAAE21B
:10108000B1E0882780F98C9308950E94D60C13EC68
:101090000E94EE0C0E940B0DAFE0B1E01C930E9489
:1010A000E50C62FAAAE2B1E0882780F98C930895F2
:1010B0000E94D60C18E60E94EE0CABE0B1E011964F
:1010C0008C91A9E0B1E08D9388278C93A9E0B1E0E1
:1010D0001C910E94EE0CABE0B1E08C91A9E0B1E074
:1010E0008D9388278C93A9E0B1E01C910E94EE0CAF
:1010F00082E0A9E0B1E08D9388278C93A9E0B1E06C
:101100001C910E94EE0C88E5A9E0B1E08D93882740
:101110008C93A9E0B1E01C910E94EE0C0E94E50CBA
:1011200062FAAAE2B1E0882780F98C9308950091D1
:101130002801013011F00C949F080C94A90802308A
:1011400011F00C94A5080C94A908033011F00C942C
:10115000A908089570916F007E7F70936F00E998E1
:1011600000912901013011F00C94B908E99A0C940E
:10117000C208023011F00C94C20870916F007160C7
:1011800070936F0008950F921F922F923F924F928B
:101190005F927F92AF92BF920F931F932F933F93D3
:1011A0004F935F936F937F938F939F93AF93BF936F
:1011B000CF93DF93EF93FF938FB78F9380EE80935E
:1011C000850080EC80938400A9E2B0E00C9103FBE1
:1011D00081E00EF080E08F93A9E2B0E00C9102FB79
:1011E00081E00EF080E09F918923882311F40C9414
:1011F000FE0870910001706270930001A9E2B0E0F6
:101200000C9103FB81E00EF480E08F93A9E2B0E043
:101210000C9102FB81E00EF480E09F9189238823EA
:1012200011F40C941809709100017F7D70930001F6
:10123000A9E2B0E00C9103FB81E00EF480E08F9313
:10124000A9E2B0E00C9102FB81E00EF080E09F91FA
:101250008923882311F40C94320970910001706184
:1012600070930001A9E2B0E00C9103FB81E00EF065
:1012700080E08F93A9E2B0E00C9102FB81E00EF4D4
:1012800080E09F918923882311F40C944C0970917C
:1012900000017F7E709300010027A0E0B1E08C91F7
:1012A00085FB00F94427A0E0B1E08C9183FB40F975
:1012B000041711F40C94AE09A0E0B1E08C9185FB09
:1012C00081E00EF080E08F93A0E0B1E08C9184FB90
:1012D00081E00EF080E09F918923882311F40C9423
:1012E0007B0970910001706870930001709100019A
:1012F0007F7B70930001A0E0B1E08C9185FB81E0E1
:101300000EF480E08F93A0E0B1E08C9184FB81E04B
:101310000EF080E09F918923882311F40C949A09A0
:10132000709100017F7770930001709100017064EB
:1013300070930001A0E0B1E08C9185FBA0E0B1E0EA
:101340008C9183F98C9380E080932601A5E2B1E033
:101350000C9101FB16F00C94AE092C9A4C990C944C
:10136000BC0980E080932601A5E2B1E00C9101FB6D
:1013700016F00C94BC092C9A8F918FBFFF91EF91BE
:10138000DF91CF91BF91AF919F918F917F916F919D
:101390005F914F913F912F911F910F91BF90AF900F
:1013A0007F905F904F903F902F901F900F901895D7
:1013B0000F921F922F923F924F925F927F92AF9225
:1013C000BF920F931F932F933F934F935F936F930E
:1013D0007F938F939F93AF93BF93CF93DF93EF93BD
:1013E000FF938FB78F934A9B0C94120A4B9B0C94DC
:1013F000030A709100017064709300017091000104
:101400007F77709300014B990C94100A7091000142
:10141000706870930001709100017F7B70930001F0
:101420000C942C0A4B9B0C941F0A7091000170685D
:1014300070930001709100017F7B709300014B99C4
:101440000C942C0A709100017064709300017091EB
:1014500000017F777093000181E090E00E94F30B20
:1014600080E080932601A5E2B1E00C9101FB16F02B
:101470000C943B0A2C9A8F918FBFFF91EF91DF91D3
:10148000CF91BF91AF919F918F917F916F915F911C
:101490004F913F912F911F910F91BF90AF907F90EF
:1014A0005F904F903F902F901F900F9018950F9244
:1014B0001F922F923F924F925F927F92AF92BF9274
:1014C0000F931F932F933F934F935F936F937F934C
:1014D0008F939F93AF93BF93CF93DF93EF93FF933C
:1014E0008FB78F93809126018150809326010091C0
:1014F0002601003011F00C94850AA5E2B1E00C91B0
:1015000002FB16F40C94850A2C988F918FBFFF91E3
:10151000EF91DF91CF91BF91AF919F918F917F918B
:101520006F915F914F913F912F911F910F91BF90BC
:10153000AF907F905F904F903F902F901F900F90B3
:10154000189509D00E94020C00FC10D0089503D019
:101550001ED001F8F9CF0024E89457FF02C009D04B
:10156000689400F80BD010F80124089502D009D037
:101570000895509540954F5F5F4F0895E89417FF89
:101580000895009510950F5F1F4F68940895352FAB
:10159000242FE894452B11F468940895512F402F7F
:1015A0000027112780E1440F551F001F111F021B48
:1015B000130B416018F4020F131F4E7F8A9599F7A1
:1015C00008958F938D918823E9F711978F9108954E
:1015D00088270090C00007FE089500C08091C000D9
:1015E00087FFFCCF8091C6000895A8E9B4E08D91F3
:1015F000882311F06ED0FBCF08950E94350C802D0A
:1016000011F067D0FACF089580EC69C081E067D00F
:1016100015D080E864C08FE7213039F08FEB22309D
:1016200021F08FE8233009F08FEC810F0C946F0BC1
:1016300088EE93E0D8D03197D9F7089583E09927C1
:10164000D2C08AEF90E00E94F30B239A229A219A4B
:10165000209A279A269A2E9885E090E00E94F30B14
:101660002F982B982A98299A289A2F9AEF93FF93CC
:10167000E4ECF0E00E94E70BFF91EF912F98B0D0DF
:101680002F9AEF93FF93E4ECF0E00E94E70BFF91B9
:10169000EF912F98A5D02F9AEF93FF93E4ECF0E011
:1016A0000E94E70BFF91EF912F989AD028982F9ADC
:1016B000EF93FF93E4ECF0E00E94E70BFF91EF91D2
:1016C0002F988ED088E20BD08EE009D086E007D02C
:1016D00008952E9A829505D004D082D008952E9830
:1016E000F9CF859510F4289A01C02898859510F4B3
:1016F000299A01C02998859510F42A9A01C02A9840
:10170000859510F42B9A01C02B982F9AEF93FF9395
:10171000E4ECF0E00E94E70BFF91EF912F98089521
:1017200000FC05D0089530D005D001F8F9CF37D0AE
:101730003FD00895842F952FA62FB72FE894452BDF
:10174000462B472B11F468940895402F512F622F98
:10175000732F0027112722273327F0E2440F551F4C
:10176000661F771F001F111F221F331F081B190B35
:101770002A0B3B0B416028F4080F191F2A1F3B1F3F
:101780004E7FFA9559F708950024E89477FF02C038
:1017900006D0689400F809D010F80124089512D0FA
:1017A0004F5F5F4F6F4F7F4F0895E89437FF089565
:1017B00000951095209530950F5F1F4F2F4F3F4F8D
:1017C0006894089540955095609570950895319767
:1017D000F1F70895689462F80895E89462F808951E
:1017E00081E090E000C0EF93FF93EE27E82BE92B18
:1017F00031F0E0EDF7E03197F1F70197D1F7FF9184
:10180000EF9108950F92B801469F8001479F100DF8
:10181000569F100D0F9008950F921F922F92C8019E
:10182000D901489F80014A9F90014B9F202C499FDE
:10183000100D211D321D5A9F202C589F100D211D67
:10184000321D599F200D311D689F200D311D699F4C
:10185000300D789F300D2F901F900F9008950E94AB
:10186000350C0D920020D9F70895C89531960020C7
:101870000895000F111F221F331F08950095109522
:10188000209530950F5F1F4F2F4F3F4F08950191C7
:1018900010810EC001911191219130810BC00191F5
:1018A000108117FF05C03FEF2FEF04C00081112703
:1018B0002227332737FF03C0E1DF8DE28D93CF93DB
:1018C000DF93CF92DF92EF92AA24BB24CC24DD24B5
:1018D000EE2440E2CAE0DD2755E093E38881890FDA
:1018E00087FD9F7083FD907F891B89935A95A9F787
:1018F000C0DFAA1CBB1CCC1CDD1CEE1C4A9551F79A
:10190000E894EFE0FF2782910ED0EB30E0F71EF075
:1019100068948A2D0CD088278D93EF90DF90CF901C
:10192000DF91CF910895982F829501D0892F8F70E4
:10193000805D26F0803309F4089568948D930895AE
:10194000F999FECFE1BDF2BD3196089591E001C055
:1019500092E07B3751F47FB7F894F2DF8D9180BD30
:10196000FA9AF99A9A95C9F77FBF7727089591E077
:1019700001C092E0E5DFF89A80B58D939A95D1F792
:101980000895FF93881BF9E0001FFA9511F4FF9169
:101990000895881F841B18F4840F8894F5CF089449
:1019A000F3CF449845983C983D9808953D9A3C98CB
:1019B00003D03D9801D03C9AEF93FF93E6E0F0E02E
:1019C0000E94E70BFF91EF9108953D9A3C9AF4DF56
:1019D0003D98359BFECFF0DF3C98EECF0894111F69
:1019E00001C0110F69F03D9A18F400003C9802C044
:1019F0003C9A00C0E1DF3D98359BFECFDDDFF1CFA3
:101A00003D9A3C98D9DF3D98359BFECFE8943499B8
:101A1000689462F8D1CF089401C08894331F11E014
:101A20003D9A3C98C9DF3D98359BFECFC5DF889431
:101A300034990894111FA0F73D9A379510F43C98FB
:101A400001C03C9AB9DF3D98359BFECFB5DF0895C4
:101A50004154562D54580000205630316500444CF6
:101A6000314D464B2031312F3230313200004C4362
:101A7000442D5479700045004C005800536368723F
:101A80006974747765697465000056657276696576
:101A90006C66616368756E6700004C6F636B6269AA
:101AA00074004C43442D42656C6575636874756EB3
:101AB0006700546F6E747284676572004672657158
:101AC00075656E7A616E7A65696765006B487A0044
:101AD00020002D66616368004175730045696E00E2
:101AE0004461756572004472656867656265722D50
:101AF000547970004578697420496E6974003136F4
:101B0000202A203100003136202A20316100313670
:101B1000202A20320000547970200000506F6C6C35
:101B2000696E000050616E61736F6E6963002E0014
:0C1B300030004D487A00537465702000AE
:00000001FF
